:020000040801F1
:107000001C491B4808601D491B4808601D491C4855
:1070100008601E491C4808601E491D4808601F4939
:107020001D4808601F491E48086020491E48086026
:1070300020491F48086021491F480860214920480D
:1070400008602249204808602249214808602349F5
:1070500021480860234922480860244922480860E2
:1070600024492348086025492348086070470000E8
:10707000197C01083C0700202B7401084007002000
:10708000CF730108F405002051730108F8050020B2
:1070900021730108FC0500209772010800060020FA
:1070A000957201080406002093720108080600206A
:1070B00091720108100600208F720108140600204A
:1070C0008D72010844070020917101080C06002010
:1070D0004B7101081806002049710108480700207B
:1070E000477101081C060020452C000820060020DE
:1070F00001710108240600205204002038070020F6
:10710000FE4810B500780022FD49012806D0FD4850
:10711000007878B101280FD002280FD00A70FB4AFE
:10712000F94C0978126820789047207848B10020FF
:10713000207010BD102002E00F2000E00D2008702C
:10714000EDE70120F4E77047704770472DE9F04103
:10715000EF480178EF48006811B1C0F3470600E03E
:10716000C6B2ED48ED4D4FF47A780478EC4F07E065
:10717000396840468847296830468847641EE4B22B
:10718000002CF5D1E74829680068BDE8F0410847C0
:1071900070B5E54DDD4C687828B11A2122680020D1
:1071A0009047FFF7D3FFA87928B11B212268002060
:1071B0009047FFF7CBFFE87928B11921226800201A
:1071C0009047FFF7C3FF287A28B11D2122680020CD
:1071D0009047FFF7BBFF687A28B11E212268002084
:1071E0009047FFF7B3FF687928B11C21226800207F
:1071F0009047FFF7ABFFA87A28B122212268002030
:107200009047FFF7A3FFE87A28B1212122680020E8
:107210009047FFF79BFFE87828B1202122680020E3
:107220009047FFF793FF287928B11F21226800209B
:107230009047FFF78BFF287B28B1072122680020A9
:107240009047FFF783FF687B28B105212268002063
:107250009047FFF77BFFA87B28B10621226800201A
:107260009047FFF773FFE87B28B1242122680020B4
:107270009047FFF76BFFA878002806D023212268EB
:1072800000209047BDE8704060E770BD70477047D0
:1072900070477047704770B59C4C082101202268E8
:1072A000904710212268012090470F212268012079
:1072B00090470D2122680120904718212268012063
:1072C00090471721226801209047984D984AFA204C
:1072D00028600821126800209047904E2868316885
:1072E0008847122122680120904792480068804711
:1072F00012212268002090473168286888478E480C
:10730000007800280BD00320ECF74BF87D4908707B
:107310008B498A48096888478A490020087070BDEF
:1073200070B5894E292031688847884C804D20707F
:1073300008B1062106E031682A208847207000281D
:1073400005D007212A68BDE870400020104770BDB5
:107350007F490020804A08707E4908707249087091
:10736000107048708870C870087148718871C87151
:10737000087248728872C87208734873774A8873B3
:10738000C8731070764A1070764A10700874764987
:10739000764A087001211170754A1070754A1060A4
:1073A000754A11705C4A1170744A1070744A10600A
:1073B000744A11707449086074490870744908600F
:1073C00074490870744908707449087070477449AA
:1073D0000020744A087001211170734A1070734ABA
:1073E0001070734A1070734A1060734A1070734AB9
:1073F0001060734A1060734A1070734A1060734AC9
:107400001060734A1070734A1060734A1060734AB8
:107410001070734A1060734A1170744A7249116097
:1074200073490870734908607047734910B50520A7
:10743000087072490F20354C087071491A20087085
:1074400070480021017015214170162181701421AE
:10745000C170132101716C49012008706B490870DB
:1074600022680821904710212268012090470F21AF
:107470002268012090470D212268012090471821A1
:1074800022680120904722681721BDE810400120A2
:1074900010475F4910B540F6B830086020490968C8
:1074A000884721484178002926D08178002923D0B7
:1074B000C178002920D0017900291DD04179002907
:1074C0001AD08179002917D0C179002914D0017A06
:1074D000002911D0417A00290ED0817A00290BD0E1
:1074E000C17A002908D0017B002905D0417B002901
:1074F00002D0817B00298DE09FE0000095050020EF
:10750000820500209605002093050020A804002095
:10751000C30300202804002066050020E4040020A6
:10752000D404002030040020400400209C050020EA
:107530009C04002074040020CE030020D406002008
:10754000C004002094050020F004002073050020F2
:1075500031070020320700203307002035070020C4
:107560002A070020360700202F070020630500208F
:1075700064050020980500206505002067050020AF
:107580002007002028070020A00500202907002050
:107590001C07002068050020690500206A050020FE
:1075A0006B0500206C0500206E0500206F05002093
:1075B00070050020B00500202B070020B405002036
:1075C000B80500202C070020BC050020C0050020C5
:1075D0002D070020C4050020C80500202E0700202C
:1075E000CC0500207105002040420F00D00500208E
:1075F0007205002024070020880500208305002054
:10760000600500202C0600207D0500207E0500205E
:10761000D405002011D0C17B00290ED001210170BA
:10762000FE48FF4C01700E2122680120904722681D
:107630000921BDE810400120104710BDF94810B5E0
:10764000C179002909D10121F54AC17119211268B6
:1076500001209047BDE810401BE710BDF2493220E1
:107660000860F24909680847EE4810B58179002999
:1076700009D10121EA4A81711B211268012090473A
:10768000BDE8104005E710BDE64810B54179002976
:1076900009D10121E24A41711C2112680120904761
:1076A000BDE81040F5E610BDDE4810B501790029AF
:1076B00009D10121DA4A01711F2112680120904786
:1076C000BDE81040E5E610BDD64810B5C1780029E8
:1076D00009D10121D24AC1702021126801209047AE
:1076E000BDE81040D5E610BDCE4810B58178002920
:1076F00009D10121CA4A81702321126801209047D3
:10770000BDE81040C5E610BDC64810B5C17B0029D4
:1077100009D10121C24AC173242112680120904776
:10772000BDE81040B5E610BD10B5BE48BC4C417C6C
:10773000226839B1002141740B21002090470C21AF
:10774000012006E0012141740B21012090470C210A
:1077500000202268BDE810401047B34910B54FF42F
:10776000FA700860B14909688847B1480078002874
:1077700002D0BDE81040D7E710BD022807D003288B
:1077800007D0042807D0052807D00020704715200F
:10779000704716207047142070471320704770B54B
:1077A000A44C2078052812D2FFF7E7FF9C4D014634
:1077B00000202A6890472078401CC0B22070FFF754
:1077C000DCFF2A68BDE8704001460120104770BD0B
:1077D00010B5FFF7E4FF954941F288300968BDE82C
:1077E000104008479448904A03789048052B016858
:1077F00002D24FF47A7000E064201060084770B540
:10780000FFF7C6FC864C12210120226890478B4A64
:107810000821002012689047894D8A4EFA2028607E
:107820003168884788480068804712212268002014
:10783000904709212268002090470E2122680020ED
:10784000904778490020087448700872487288721E
:10785000C872087348738873C8738870C8700871D9
:1078600048718871C871087008212268012090470A
:1078700028683168BDE87040084710B5684C0C2195
:107880000020226890470B21226800209047684919
:10789000002008706D49012008706D480068BDE83F
:1078A0001040004710B5FFF77AFF604941F2883079
:1078B000096888475E485B4C007838B1607C18B135
:1078C0005D480078052801D2FFF7D7FF207808B17E
:1078D000FFF795FF594A072100201268BDE81040C4
:1078E000104710B5FFF75BFF504941F28830096837
:1078F00088474F484B4C007838B1607C18B94E48E7
:107900000078052801D2FFF7B8FF207808B1FFF70B
:1079100076FF4A4A062100201268BDE81040104751
:1079200070B54A480078002813D1414801253C4CE5
:10793000057041480078052803D20C2122680120F7
:10794000904738480B2145742268BDE870400120FB
:10795000104770BD70B53349314C012088732268DF
:10796000062190470821226800209047394D287849
:1079700040B13948006880470A21226800209047BA
:10798000002028703548007808B1FFF7C9FF264964
:107990004FF4FA600860254909688847BDE87040DF
:1079A00077E52F4810B50078002817D02D480078CB
:1079B000002813D02C48007800280FD02749012038
:1079C000174A08702349087012680A219047154821
:1079D000807B002802D0BDE81040A1E710BD204800
:1079E00010B5017861B901210D4C01701021226898
:1079F000002090471821226800209047FFF7D1FF10
:107A00001A48007840B11A48007828B91948007817
:107A100010B919480068804730E0000035070020A1
:107A2000A804002040040020D4050020D404002035
:107A30002F07002066050020BB0300209C040020C7
:107A40009C050020E4040020740400202907002085
:107A5000800400202A0700205C0400203607002054
:107A6000310700203207002033070020CE0300201A
:107A70006B05002096050020D8040020B84941F28B
:107A800088300968BDE810400847B64810B501784D
:107A900061B90121B44C01700D212268002090478A
:107AA0001721226800209047FFF77BFFAF4800783E
:107AB00048B1AF48007830B9AE480078022802D10A
:107AC000AD4800688047AD4941F288300860A4495C
:107AD0000968BDE81040084710B5A94C207840B9A6
:107AE000A14A0F2100201268904701202070FFF763
:107AF00058FF9E48007848B19D48007830B99D48AD
:107B00000078012802D19C4800688047944941F2DE
:107B100088300968BDE8104008479A4810B5417B95
:107B2000002909D10121904A4173052112680120E1
:107B30009047BDE81040ACE410BD904910B50A2054
:107B400008608749096888478F480078002802D074
:107B5000BDE81040E8E510BD8A4810B5017B00295A
:107B600009D10121804A0173072112680120904741
:107B7000BDE810408DE410BD824810B5C17A0029DF
:107B800009D10121784AC172212112680120904750
:107B9000BDE810407DE410BD7A4810B5817A002917
:107BA00009D10121704A8172222112680120904777
:107BB000BDE810406DE410BD724810B5417A00294F
:107BC00009D10121684A41721E21126801209047A3
:107BD000BDE810405DE410BD6A4810B5017A002987
:107BE00009D10121604A01721D21126801209047CC
:107BF000BDE810404DE410BD624810B54178002941
:107C000009D10121584A41701A2112680120904778
:107C1000BDE810403DE410BD10B5292861D01BDC43
:107C200017284CD00BDCA0F10A000C2832D2DFE878
:107C300000F03437313A3D31313131314043202881
:107C400046D004DC18283DD01E2823D13DE0222850
:107C500041D028281ED141E03F2857D00EDC3628DD
:107C60004BD006DC2A283FD0322840D0352811D10D
:107C700040E03C2844D03D280CD144E047284ED079
:107C800004DC402845D0462804D145E0492849D0A5
:107C90004A284AD04FF0FF3010BDFFF7ADFF46E055
:107CA000FFF79AFF43E0FFF787FF40E0FFF774FF1D
:107CB0003DE0FFF761FF3AE0FFF74EFF37E0FFF7E7
:107CC0003CFF34E0FFF729FF31E0FFF705FF2EE02E
:107CD000FFF7DBFE2BE0FFF782FE28E0FFF73AFE1E
:107CE00025E0FFF7FEFD22E0FFF7DCFD1FE0FFF7D8
:107CF00079FD1CE0FFF76CFD19E0FFF72EFD16E0A3
:107D0000FFF702FD13E0FFF7EFFC10E0FFF7DCFCEC
:107D10000DE0FFF7C9FC0AE0FFF7B6FC07E0FFF74C
:107D2000A3FC04E0FFF79AFC01E0FFF787FC0020CA
:107D300010BD7047154801781048012902D1144937
:107D40000968016013490068086014491248086016
:107D5000144913480860144942F2107008607047D3
:107D6000D404002033070020A8040020CE03002004
:107D70006B05002096050020D8040020D4050020C3
:107D800032070020400400202F0700207905002042
:107D9000E0050020DC05002080380100EC05002013
:0C7DA000301B0F00E8050020E405002067
